:10000000B4010529A501A400B5172730A3001030BD
:1000100015200330A300E8301520A301643015201B
:10002000A3010A30152024082028A2002508A100D9
:100030002408A000CE202008031DB513B51B08001E
:10004000303EA7000711871007108316071187108D
:100050000710F030860583122708B4184D283A306F
:10006000A1009830A8203330A60062201330A100F0
:100070008830A82062206430A72062206430A72046
:100080002230A600622028304C200C304C20063054
:100090004C20B41427084D283414A600341C5B28C7
:1000A0008710033C031C602860200730A100D0307B
:1000B000A820031408003414FE3C031900298714F7
:1000C000A60E341C34100715F030860526080F39AB
:1000D00086040711A60E341862283230A7200314B4
:1000E0000800A000A00DA00D200D383981389F0018
:1000F0000030A1003230A8201F151F197D281E08CE
:10010000A10083161E08002903178D0083168C1387
:100110000C1483120C08002903178C0083168C130F
:100120000C1555308D00AA308D008C148C18962833
:100130000C110029A301A200FF30A207031CA30792
:10014000031C00290330A100E630A8209C28A1014F
:10015000FC3EA000A109031CB328FF300000A0074B
:100160000318AE28A0076400A10FAD280800A20064
:100170000130BE28A301A2000430BE28A800230835
:100180002102031DC5282208200204300318013073
:10019000031902302805031DFF300029A501A40121
:1001A0001030A600210DA40DA50D2208A4022308DD
:1001B000031C230FA5020318E4282208A407230820
:1001C0000318230FA5070310A00DA10DA60BD2281D
:1001D000200800291030A800A101A001A70CA60C3E
:1001E000031CF8282208A00723080318230FA107DF
:1001F000A10CA00CA50CA40CA80BEE282408002927
:10020000831303138312640008008316DF30850014
:1002100082309F0070308600811387018312850130
:10022000860187018A11B429861783168613FE304A
:1002300083128A01212001308A01212054308A0151
:10024000212057308A01212043308A01212031307A
:100250008A0121202E308A01212030308A0121207C
:1002600020308A01212066308A0121206F308A01E6
:10027000212072308A01212020308A012120323051
:100280008A01212030308A0121204D308A0121202D
:1002900048308A0121207A308A0121200330A300CE
:1002A000E8308A019B20FE308A012120C0308A017B
:1002B000212050308A01212072308A0121206F30A4
:1002C0008A01212064308A01212075308A01212091
:1002D00063308A01212065308A01212064308A013F
:1002E000212020308A01212062308A0121207930AA
:1002F0008A01212020308A01212049308A012120D1
:100300007A308A01212075308A0121200730A3002C
:10031000D0308A019B20080003308A017120BA0086
:100320002108BB000A308A019A20080002308A01A5
:100330007120BE002108BF000A308A019A200800FF
:1003400001308A017120C2002108C3000A308A01ED
:100350009A20080000308A017120C6002108C700D9
:100360000A308A019A2008000713831607138312A4
:1003700007128316071283128711831687118312BF
:1003800085128316851283128A0114213F30CE0014
:100390003F30CF003F30D0003F30D10005308A01E0
:1003A0008420D30006308A018420D40007308A01DB
:1003B0008420D50008308A018420D60009308A01C3
:1003C0008420D7000A308A018420D8000B308A01AB
:1003D0008420D9000C308A018420DA000D308A0193
:1003E0008420D2005208A600A7010A30A200A3016F
:1003F0008A01EA20CC002508CD00CA01CB01861372
:1004000083168613FE3083128A01212001308A016F
:10041000212053088A0102203A308A012120540801
:100420008A0102203A308A01212055088A010220DF
:100430003A308A01212056088A0102203D308A0183
:10044000212052088A01022030308A012120FE300A
:100450008A012120C0308A01212057088A01022008
:100460003A308A01212058088A0102203A308A0154
:10047000212059088A0102203A308A0121205A0895
:100480008A01022020308A0121204F308A01212058
:100490004B308A0121203F308A0121200130A30006
:1004A0002C308A019B20071383160713831207122F
:1004B0008316071283128711831687118312851200
:1004C0008316851264008A118312061ECA2F6400E7
:1004D0008A11861E6D2A8A01532A64308A019A2065
:1004E00064008A11861E6D2AFE308A0121200130A7
:1004F0008A01212053308A01212045308A012120A0
:1005000054308A01212020308A01212048308A017C
:10051000212069308A01212020308A012120543095
:100520008A01212045308A0121204D308A01212075
:1005300050308A01212020308A01212041308A0157
:1005400021203D308A01212053088A010220FE30FB
:100550008A012120C0308A01212052308A012120C5
:100560003A308A0121204E308A01212065308A01EB
:10057000212078308A01212074308A012120203006
:100580008A01212059308A0121203A308A01212014
:1005900044308A0121206E308A01212020308A01D6
:1005A000212042308A0121203A308A012120553011
:1005B0008A01212070308A01212064308A019A202A
:1005C00064008A11061AE52AD30A640060305302D7
:1005D0008A11031CED2A5F30D30064008A11861A49
:1005E000F22AD30364000A3053028A110318FA2A4C
:1005F0000A30D30064008A11061F002B8A01742A76
:1006000064308A019A2064008A11061F002BFE3094
:100610008A01212001308A01212053308A012120C2
:1006200045308A01212054308A01212020308A015E
:10063000212048308A01212069308A012120203080
:100640008A01212054308A01212045308A0121204D
:100650004D308A01212050308A01212020308A012A
:10066000212042308A0121203D308A012120540876
:100670008A010220FE308A012120C0308A01212017
:1006800052308A0121203A308A0121204E308A01DD
:10069000212065308A01212078308A0121207430A0
:1006A0008A01212020308A01212059308A0121200D
:1006B0003A308A01212044308A0121206E308A019B
:1006C000212020308A01212042308A0121203A3025
:1006D0008A01212055308A01212070308A01212091
:1006E00064308A019A2064008A11061A782BD40A91
:1006F0006400603054028A11031C802B5F30D400E8
:1007000064008A11861A852BD40364000A305402CF
:100710008A1103188D2B0A30D40064008A11061F39
:10072000932B8A01072B64308A019A2064008A1176
:10073000061F932BFE308A01212001308A012120DF
:1007400053308A01212045308A01212054308A010A
:10075000212020308A01212048308A01212069305F
:100760008A01212020308A01212054308A01212051
:1007700045308A0121204D308A01212050308A01E4
:10078000212020308A01212043308A0121203D3060
:100790008A01212055088A010220FE308A01212089
:1007A000C0308A01212052308A0121203A308A014A
:1007B00021204E308A01212065308A0121207830A5
:1007C0008A01212074308A01212020308A012120D1
:1007D00059308A0121203A308A01212044308A018F
:1007E00021206E308A01212020308A0121204230D0
:1007F0008A0121203A308A01212055308A012120A6
:1008000070308A01212064308A019A2064008A11A4
:10081000061A0B2CD50A6400603055028A11031C9D
:10082000132C5F30D50064008A11861A182CD5036A
:1008300064000A3055028A110318202C0A30D500B2
:1008400064008A11061F262C8A019A2B64308A01C3
:100850009A2064008A11061F262CFE308A0121206E
:1008600001308A01212053308A01212045308A013C
:10087000212054308A01212020308A012120483053
:100880008A01212069308A01212020308A0121201B
:1008900054308A01212045308A0121204D308A01BF
:1008A000212050308A01212020308A01212044302B
:1008B0008A0121203D308A01212056088A01022028
:1008C000FE308A012120C0308A01212052308A0165
:1008D00021203A308A0121204E308A0121206530C2
:1008E0008A01212078308A01212074308A01212058
:1008F00020308A01212059308A0121203A308A0192
:10090000212044308A0121206E308A0121202030AC
:100910008A01212042308A0121203A308A01212097
:1009200055308A01212070308A01212064308A01EB
:100930009A2064008A11061A9E2CD60A6400603040
:1009400056028A11031CA62C5F30D60064008A115F
:10095000861AAB2CD60364000A3056028A1103189B
:10096000B32C0A30D60064008A11061FB92C8A0104
:100970002D2C64308A019A2064008A11061FB92C3C
:10098000FE308A01212001308A01212048308A016D
:10099000212069308A01212020308A012120543011
:1009A0008A01212049308A0121204D308A012120ED
:1009B00045308A0121203D308A01212052088A01D8
:1009C000022030308A01212073308A0121206530D5
:1009D0008A01212063308A012120FE308A012120F2
:1009E000C0308A01212052308A0121203A308A0108
:1009F00021204E308A01212065308A012120783063
:100A00008A01212074308A01212020308A0121208E
:100A100059308A0121203A308A01212044308A014C
:100A200021206E308A01212020308A01212042308D
:100A30008A0121203A308A01212055308A01212063
:100A400070308A01212064308A019A2064008A1162
:100A5000061A2B2DD20A64008A11861A302DD20371
:100A60006400FB3052028A11031C372DD20164004E
:100A70008A11061F3D2D8A01C02C64308A019A20FC
:100A800064008A11061F3D2DFE308A0121200130AD
:100A90008A01212053308A01212045308A012120FA
:100AA00054308A01212020308A0121204C308A01D3
:100AB00021206F308A01212020308A0121205430EA
:100AC0008A01212045308A0121204D308A012120D0
:100AD00050308A01212020308A01212041308A01B2
:100AE00021203D308A01212057088A010220FE3052
:100AF0008A012120C0308A01212052308A01212020
:100B00003A308A0121204E308A01212065308A0145
:100B1000212078308A01212074308A012120203060
:100B20008A01212059308A0121203A308A0121206E
:100B300044308A0121206E308A01212020308A0130
:100B4000212042308A0121203A308A01212055306B
:100B50008A01212070308A01212064308A019A2084
:100B600064008A11061AB52DD70A6400473057026F
:100B70008A11031CBD2D4630D70064008A11861AE5
:100B8000C22DD70364000A3057028A110318CA2DF8
:100B90000A30D70064008A11061FD02D8A01442D27
:100BA00064308A019A2064008A11061FD02DFE301D
:100BB0008A01212001308A01212053308A0121201D
:100BC00045308A01212054308A01212020308A01B9
:100BD00021204C308A0121206F308A0121202030D1
:100BE0008A01212054308A01212045308A012120A8
:100BF0004D308A01212050308A01212020308A0185
:100C0000212042308A0121203D308A0121205808CC
:100C10008A010220FE308A012120C0308A01212071
:100C200052308A0121203A308A0121204E308A0137
:100C3000212065308A01212078308A0121207430FA
:100C40008A01212020308A01212059308A01212067
:100C50003A308A01212044308A0121206E308A01F5
:100C6000212020308A01212042308A0121203A307F
:100C70008A01212055308A01212070308A012120EB
:100C800064308A019A2064008A11061A482ED80A14
:100C90006400473058028A11031C502E4630D80099
:100CA00064008A11861A552ED80364000A3058024F
:100CB0008A1103185D2E0A30D80064008A11061FBD
:100CC000632E8A01D72D64308A019A2064008A112C
:100CD000061F632EFE308A01212001308A01212067
:100CE00053308A01212045308A01212054308A0165
:100CF000212020308A0121204C308A0121206F30B0
:100D00008A01212020308A01212054308A012120AB
:100D100045308A0121204D308A01212050308A013E
:100D2000212020308A01212043308A0121203D30BA
:100D30008A01212059088A010220FE308A012120DF
:100D4000C0308A01212052308A0121203A308A01A4
:100D500021204E308A01212065308A0121207830FF
:100D60008A01212074308A01212020308A0121202B
:100D700059308A0121203A308A01212044308A01E9
:100D800021206E308A01212020308A01212042302A
:100D90008A0121203A308A01212055308A01212000
:100DA00070308A01212064308A019A2064008A11FF
:100DB000061ADB2ED90A6400473059028A11031C37
:100DC000E32E4630D90064008A11861AE82ED90332
:100DD00064000A3059028A110318F02E0A30D90033
:100DE00064008A11061FF62E8A016A2E64308A0179
:100DF0009A2064008A11061FF62EFE308A012120F7
:100E000001308A01212053308A01212045308A0196
:100E1000212054308A01212020308A0121204C30A9
:100E20008A0121206F308A01212020308A0121206F
:100E300054308A01212045308A0121204D308A0119
:100E4000212050308A01212020308A012120443085
:100E50008A0121203D308A0121205A088A0102207E
:100E6000FE308A012120C0308A01212052308A01BF
:100E700021203A308A0121204E308A01212065301C
:100E80008A01212078308A01212074308A012120B2
:100E900020308A01212059308A0121203A308A01EC
:100EA000212044308A0121206E308A012120203007
:100EB0008A01212042308A0121203A308A012120F2
:100EC00055308A01212070308A01212064308A0146
:100ED0009A2064008A11061A6E2FDA0A64004730DD
:100EE0005A028A11031C762F4630DA0064008A11F8
:100EF000861A7B2FDA0364000A305A028A1103181B
:100F0000832F0A30DA0064008A11061F892F8A01B4
:100F1000FD2E031705308D00031353088A018C2022
:100F2000031706308D00031354088A018C20031721
:100F300007308D00031355088A018C2003170830F1
:100F40008D00031356088A018C20031709308D0089
:100F5000031357088A018C2003170A308D000313EE
:100F600058088A018C2003170B308D000313590891
:100F70008A018C2003170C308D0003135A088A0154
:100F80008C2003170D308D00031352088A018C202A
:100F90008A01CE29CA0A0319CB0A4A08A0004B08C5
:100FA000A1004D08A3004C088A01B7208A15031D33
:100FB0009F298A018C213A08A6003B08A7007D30B2
:100FC000A200A3018A01EA20B2002508B30032087A
:100FD000A0003308A100A2010130A3008A01CE20A5
:100FE000BC002108BD008A0196213E08A6003F08EA
:100FF000A7007D30A200A3018A01EA20B2002508E3
:10100000B3003208A0003308A100A2010130A30000
:101010008A01CE20C0002108C1008A01A021420817
:10102000A6004308A7007D30A200A3018A01EA20A0
:10103000B2002508B3003208A0003308A100A201C5
:101040000130A3008A01CE20C4002108C5008A0116
:10105000AA214608A6004708A7007D30A200A301E8
:101060008A01EA20B2002508B3003208A000330844
:10107000A100A2010130A3008A01CE20C8002108EE
:10108000C900FE308A01212001308A0121204B084D
:10109000A5004A088A01032073308A0121206530A7
:1010A0008A01212063308A01212020308A012120F9
:1010B00062308A01212079308A01212020308A0182
:1010C00021204D08A5004C088A01032073308A01B5
:1010D0002120FE308A012120C0308A0121204E08C3
:1010E0008A0121203D08A5003C088A010320203008
:1010F0008A012120FE308A012120C0308A0121206E
:10110000FE308A01212014308A012120FE308A011C
:10111000212014308A012120FE308A012120143040
:101120008A0121203A308A0121204F088A0121209A
:101130004108A50040088A01032020308A012120AF
:10114000FE308A012120C0308A012120FE308A0130
:10115000212014308A012120FE308A012120143000
:101160008A012120FE308A01212014308A012120A9
:10117000FE308A01212014308A012120FE308A01AC
:10118000212014308A012120FE308A0121201430D0
:101190008A012120FE308A01212014308A01212079
:1011A0003A308A01212050088A0121204508A500F3
:1011B00044088A01032020308A012120FE308A0160
:1011C0002120C0308A012120FE308A0121201430E4
:1011D0008A012120FE308A01212014308A01212039
:1011E000FE308A01212014308A012120FE308A013C
:1011F000212014308A012120FE308A012120143060
:101200008A012120FE308A01212014308A01212008
:10121000FE308A01212014308A012120FE308A010B
:10122000212014308A012120FE308A01212014302F
:101230008A012120FE308A01212014308A012120D8
:10124000FE308A01212014308A0121203A308A019F
:10125000212051088A0121204908A50048088A0157
:10126000032020308A01212064008A11061FCE2924
:101270003C08A0003D08A10053088A01BA208A1545
:10128000031D4A2907138316071383122D30CE003E
:101290008A15502907178316071383122B30CE00A7
:1012A0004008A0004108A10054088A01BA208A150C
:1012B000031D622907128316071283122D30CF00F7
:1012C0008A15682907168316071283122B30CF0060
:1012D0004408A0004508A10055088A01BA208A15D3
:1012E000031D7A2987118316871183122D30D000B0
:1012F0008A15802987158316871183122B30D00019
:101300004808A0004908A10056088A01BA208A1599
:10131000031D922985128316851283122D30D10068
:101320008A15982985168316851283122B30D100D1
:101330000330A300B6308A019B208A01CA2FCA0A53
:101340000319CB0A4A08A0004B08A1004630A300AD
:1013500050308A01B7208A15031D792B8A018C2110
:101360003A08A6003B08A7007D30A200A3018A012D
:10137000EA20B2002508B3003208A0003308A1001B
:10138000A2010130A3008A01CE20BC002108BD00CB
:101390008A0196213E08A6003F08A7007D30A200E2
:1013A000A3018A01EA20B2002508B3003208A00098
:1013B0003308A100A2010130A3008A01CE20C000A1
:1013C0002108C1008A01A0214208A6004308A70005
:1013D0007D30A200A3018A01EA20B2002508B300F3
:1013E0003208A0003308A100A2010130A3008A0145
:1013F000CE20C4002108C5008A01AA214608A60003
:101400004708A7007D30A200A3018A01EA20B200AC
:101410002508B3003208A0003308A100A201013062
:10142000A3008A01CE20C8002108C900FE308A012D
:10143000212001308A01212041308A0121205708D2
:101440008A0102203A308A01212042308A0121207B
:1014500058088A0102203A308A01212043308A014B
:10146000212059088A0102203A308A012120443083
:101470008A0121205A088A01022020308A01212075
:1014800020308A012120FE308A012120C0308A01CB
:1014900021204E088A0121203D08A5003C088A0130
:1014A000032020308A012120FE308A012120C03013
:1014B0008A012120FE308A01212014308A01212056
:1014C000FE308A01212014308A012120FE308A0159
:1014D000212014308A0121203A308A0121204F082E
:1014E0008A0121204108A50040088A0103202030FC
:1014F0008A012120FE308A012120C0308A0121206A
:10150000FE308A01212014308A012120FE308A0118
:10151000212014308A012120FE308A01212014303C
:101520008A012120FE308A01212014308A012120E5
:10153000FE308A01212014308A012120FE308A01E8
:10154000212014308A012120FE308A01212014300C
:101550008A0121203A308A01212050088A01212065
:101560004508A50044088A01032020308A01212073
:10157000FE308A012120C0308A012120FE308A01FC
:10158000212014308A012120FE308A0121201430CC
:101590008A012120FE308A01212014308A01212075
:1015A000FE308A01212014308A012120FE308A0178
:1015B000212014308A012120FE308A01212014309C
:1015C0008A012120FE308A01212014308A01212045
:1015D000FE308A01212014308A012120FE308A0148
:1015E000212014308A012120FE308A01212014306C
:1015F0008A012120FE308A01212014308A01212015
:101600003A308A01212051088A0121204908A50089
:1016100048088A01032020308A01212064008A11B1
:10162000061FCE293C08A0003D08A10057088A01EA
:10163000BA208A15031D242B071383160713831260
:101640002D30CE008A152A2B071783160713831215
:101650002B30CE004008A0004108A10058088A01A4
:10166000BA208A15031D3C2B07128316071283121A
:101670002D30CF008A15422B0716831607128312CE
:101680002B30CF004408A0004508A10059088A016A
:10169000BA208A15031D542B8711831687118312D4
:1016A0002D30D0008A155A2B871583168711831287
:1016B0002B30D0004808A0004908A1005A088A0130
:1016C000BA208A15031D6C2B85128316851283128E
:1016D0002D30D1008A15722B851683168512831240
:1016E0002B30D1000330A300B6308A019B208A152D
:1016F0009F290713831607138312071283160712F5
:10170000831287118316871183128512831685121F
:10171000FE3083128A01212001308A0121202130EC
:101720008A01212020308A0121204F308A01212086
:1017300056308A01212045308A01212052308A0109
:10174000212020308A01212035308A0121202030BB
:101750008A01212048308A0121204F308A0121202E
:1017600055308A01212052308A01212020308A01FF
:10177000212021308A01212021308A012120FE30C0
:101780008A012120C0308A01212023308A012120B2
:1017900023308A01212023308A01212020308A0130
:1017A000212043308A01212055308A0121205430E4
:1017B0008A01212020308A0121204F308A012120F6
:1017C00046308A01212046308A01212020308A01BA
:1017D000212023308A01212023308A012120233037
:1017E0008A012120861383168613831264008A11CE
:0E17F000061FCE298A15F62B63008A15FC2BE6
:02400E00763DFD
:10420A0046004600460046001E001E001E001E0014
:02421A000C0096
:00000001FF
